:100000000C945C000C948B060C94B8060C94840041
:100010000C9484000C9484000C9484000C94840050
:100020000C9484000C9484000C9484000C94840040
:100030000C9484000C9484000C9484000C94840030
:100040000C94E5060C9484000C9445090C948400EF
:100050000C9484000C9484000C9484000C94840010
:100060000C9484000C948400000024272A000025AE
:10007000282B000023262904040404040404040299
:100080000202020202030303030303010204081035
:100090002040800102040810200102040810200002
:1000A0000000070002010000030406000000000039
:1000B00000000000F401770511241FBECFEFD4E04B
:1000C000DEBFCDBF11E0A0E0B1E0EAE1F4E102C0A3
:1000D00005900D92AC33B107D9F712E0ACE3B1E073
:1000E00001C01D92A331B107E1F710E0C8EBD0E0E9
:1000F00004C02297FE010E94070AC43BD107C9F73A
:100100000E9470050C940B0A0C940000FC011082F4
:100110008FEF81831382128282E2848386E9858352
:10012000178216820895EF92FF920F931F93CF9339
:10013000DF93EC019B0177FF03C020E030E005C0B6
:10014000653B710514F024EB30E02983EC806D8170
:1001500070E06E197109882777FD8095982F982F88
:10016000872F762F662730E040E050E00E9482091A
:1001700024EB30E040E050E00E94D609FF2400E08C
:1001800010E0102F0F2DFE2CEE24E20EF31E041FA4
:10019000151FC801B70120E430E040E050E00E94A4
:1001A000D6093B832A83DF91CF911F910F91FF9056
:1001B000EF9008955F926F927F928F929F92AF928D
:1001C000BF92CF92DF92EF92FF920F931F93DF9334
:1001D000CF93CDB7DEB76DB67EB6ADB65EB60E9434
:1001E000550720913E0130913F01409140015091CF
:1001F0004101621773078407950750F02C5E3F4F4B
:100200004F4F5F4F621773078407950708F4AFC01D
:1002100060933E0170933F018093400190934101B0
:10022000E0913C01F0913D01BB2408C082819381A3
:10023000892B09F0B3940680F781E02D3097B1F750
:10024000BB2009F494C08B2D90E0880F991F2DB727
:100250003EB7281B390B0FB6F8943EBF0FBE2DBF1B
:10026000CDB6DEB60894C11CD11CA0913C01B09162
:100270003D0120E013C012968D919C911397892B1C
:1002800049F0E22FF0E0EE0FFF1FEC0DFD1DB183F2
:10029000A0832F5F16960D90BC91A02D109759F753
:1002A0002CC0812F90E07C01EE0CFF1CEC0CFD1C9F
:1002B000D7016D917C91FC013197EE0FFF1FEC0D82
:1002C000FD1D40815181DB0112962D913C911397C8
:1002D000DA0112968D919C9113972817390730F403
:1002E000D7014D935C937183608301E01F5F1B1501
:1002F000C0F2002311F410E011C011E000E0F7CFCC
:10030000E12FF0E0EE0FFF1FEC0DFD1D0190F081DD
:10031000E02D61E080810E943D081F5F1B1580F386
:10032000F6B4EE2400E010E08F2C99241EC0EE2DD0
:10033000F0E0EE0FFF1FEC0DFD1D0190F081E02DB0
:1003400022813381280D391D86B58F1510F4005098
:100350001F4FF82EC8018F0D911D28173907A0F7E0
:1003600060E080810E943D08E394EB1400F38A2D45
:10037000952D9C010FB6F8943EBF0FBE2DBF0FB652
:10038000F8947EBE0FBE6DBECF91DF911F910F918D
:10039000FF90EF90DF90CF90BF90AF909F908F90A5
:1003A0007F906F905F9008950F931F938C01FC01D5
:1003B00060838FEF81831382128280913C01909140
:1003C0003D019783868310933D0100933C0160E0DB
:1003D00080810E943D0861E0F80180810E941F0831
:1003E00081E01F910F91089582E491E00E948600C0
:1003F0008AE491E00E94860082E591E00E948600F6
:100400000895BC018AE491E00E9493000895BC0124
:1004100082E491E00E9493000895EF92FF920F937F
:100420001F930E94DA008DE791E00E9485058823E2
:1004300009F45CC08DE791E00E948205282F80932B
:100440006401803F39F481E090E0909372018093E1
:1004500071010BC08091710190917201019749F473
:1004600080917B0190917C01019690937C01809317
:100470007B0180917B0190917C0182309105B1F4E8
:10048000422F50E09A01E4E035952795EA95E1F78F
:1004900080915A0190915B0128173907F9F44F7048
:1004A000507050937A014093790120C00397F1F482
:1004B000422F50E09A0174E0359527957A95E1F73F
:1004C00080915A0190915B012817390739F44F70D8
:1004D0005070509374014093730108C010927201E0
:1004E0001092710110927C0110927B0180917B012E
:1004F00090917C01039709F0A1C1809171019091C5
:100500007201019709F09AC110927C0110927B014F
:1005100010927201109271016AE070E080E090E048
:100520000E9463078091790190917A01843091054E
:1005300009F434C18530910594F48130910509F4B2
:1005400094C0823091051CF4892BC9F077C18230A8
:10055000910509F400C1039709F070C108C1863004
:10056000910509F44EC1863091050CF423C1873002
:10057000910509F452C1099709F060C15AC18091EF
:100580007301909174018730910509F449C0883056
:100590009105ACF483309105B9F1843091054CF4A8
:1005A0008130910539F1823091055CF5892BF9F0A4
:1005B00050C08530910571F106977CF528C08B30CD
:1005C0009105B9F18C30910534F48930910559F1D8
:1005D0000A9764F525C08D30910589F18D3091051C
:1005E0005CF18E30910571F10F9799F52EC084EB77
:1005F00090E002C084E690E09093760180937501CC
:1006000028C08AE590E0F8CF80E590E0F5CF86E459
:1006100090E0F2CF8CE390E0EFCF82E390E0ECCF7C
:1006200086E290E0E9CF89E190E0E6CF8FE090E0CC
:10063000E3CF8AE090E0E0CF88E090E0DDCF86E095
:1006400090E0DACF83E090E0D7CF1092760110925D
:10065000750160E080912F010E943D088091750135
:10066000909176010E940102E9C0809173019091FE
:1006700074018730910509F447C088309105ACF4C6
:1006800083309105A9F1843091054CF481309105B6
:1006900049F1823091054CF5892BF9F050C0853035
:1006A000910561F106976CF526C08B309105A9F193
:1006B0008C30910534F48930910549F10A9754F54D
:1006C00023C08D30910579F18D3091054CF18E303C
:1006D000910561F10F9799F52CC010927801109255
:1006E00077012DC083E090E026C086E090E023C033
:1006F00088E090E020C08AE090E01DC08FE090E0AC
:100700001AC089E190E017C086E290E014C082E34D
:1007100090E011C08CE390E00EC086E490E00BC046
:1007200080E590E008C08AE590E005C084E690E0AE
:1007300002C084EB90E0909378018093770160E0B1
:1007400080912F010E943D0880917701909178015E
:100750000E94070273C08091730190917401019708
:1007600011F461E001C060E080911F0165C060E0AC
:1007700080912F010E943D08809173019091740136
:100780002BE030E0829FB001839F700D929F700D2F
:10079000112482E591E00E94930050C08091730182
:1007A00090917401019711F461E001C060E08091C3
:1007B0002D0142C020917301309174012130310527
:1007C000A9F484E690E090936E0180936D013093DC
:1007D000700120936F010E94550760936901709327
:1007E0006A0180936B0190936C0128C01092700194
:1007F00010926F0160E070E080911D010E94C707B8
:100800001DC08091730190917401019711F461E012
:1008100001C060E080911B010FC080917301909135
:100820007401019711F461E001C060E080912B0137
:1008300003C061E080912F010E943D080E9455078E
:100840009B01AC0160936501709366018093670121
:100850009093680180916F0190917001019709F068
:1008600053C08091690190916A01A0916B01B09190
:100870006C01281B390B4A0B5B0B80916D01909129
:100880006E01AA2797FDA095BA2F281739074A07A6
:100890005B07A0F16FEF70E080911D010E94C70718
:1008A000E0906501F0906601009167011091680188
:1008B0008091690190916A01A0916B01B0916C01E6
:1008C000A8019701281B390B4A0B5B0B80916D0126
:1008D00090916E01880F991FAA2797FDA095BA2FB6
:1008E000281739074A075B0778F0E0926901F09210
:1008F0006A0100936B0110936C0106C060E070E028
:1009000080911D010E94C7071F910F91FF90EF90EA
:10091000089540E05BE460E070E08DE791E00E94C4
:10092000880564E670E080E090E00E94630760E084
:1009300070E080911D010E94C707609131017091A4
:10094000320182E491E00E94D40160913301709100
:1009500034018AE491E00E94D401609121017091F8
:10096000220182E591E00E94D40161E080912F0193
:100970000E943D086DE570E082E591E00E949300E1
:1009800061E080911B010E941F0861E080911D01C0
:100990000E941F0861E080911F010E941F0860E013
:1009A0008EE00E941F0860E08FE00E941F0860E058
:1009B00080E10E941F0860E081E10E941F0861E061
:1009C0008EE00E943D0861E08FE00E943D0861E0FA
:1009D00080E10E943D0861E081E10E943D08809134
:1009E00023010E948808892B39F081E090E09093E0
:1009F0005D0180935C0104C010925D0110925C0166
:100A0000809125010E948808892B39F082E090E0CE
:100A100090935F0180935E0104C010925F01109279
:100A20005E01809127010E948808892B39F084E0BB
:100A300090E0909361018093600104C01092610185
:100A400010926001809129010E948808892B39F059
:100A500088E090E0909363018093620104C010925B
:100A600063011092620180915E0190915F0120917B
:100A70005C0130915D01820F931F209160013091E4
:100A80006101820F931F2091620130916301820FF7
:100A9000931F90935B0180935A0160E071E08DE7B2
:100AA00091E00E948D0560915A0170915B018DE784
:100AB00091E00E947B0660E080911F010E943D084A
:100AC00061E080912F010E943D0860E080912B0140
:100AD0000E943D0860E080912D010E943D0808952C
:100AE0000E948D070E9489040E940D02FDCF89E3B8
:100AF00091E090937E0180937D010895862F0E945E
:100B00000D0908950E94260908950E941509089567
:100B1000CB01BA010E94D40808950F931F93CF937D
:100B2000DF938C01EB0109C02196D801ED91FC9176
:100B30000190F081E02DC801099568816623A1F735
:100B4000DF91CF911F910F9108950F931F938C0107
:100B5000DC01ED91FC910190F081E02D6DE00995B3
:100B6000D801ED91FC910190F081E02D6AE0C8017F
:100B700009951F910F9108952F923F924F925F9286
:100B80006F927F928F929F92AF92BF92CF92DF929D
:100B9000EF92FF920F931F93DF93CF93CDB7DEB702
:100BA000A0970FB6F894DEBF0FBECDBF1C016A013F
:100BB0007B01411551056105710549F4DC01ED9199
:100BC000FC910190F081E02D60E3099554C08824E8
:100BD00099245401422E55246624772401E010E024
:100BE0000C0F1D1F080D191DC701B601A3019201AD
:100BF0000E94B409F80160830894811C911CA11C17
:100C0000B11CC701B601A30192010E94B409C90138
:100C1000DA016C017D01C114D104E104F104F1F6A3
:100C200081E0E82EF12CEC0EFD1EE80CF91C3E01D3
:100C30000894611C711CD501C4010197A109B10977
:100C40006C01C818D90814C0F601EE0DFF1D6081B3
:100C50006A3010F4605D01C0695CD101ED91FC91D6
:100C60000190F081E02DC10109950894E108F10897
:100C70006E147F0449F7A0960FB6F894DEBF0FBE3E
:100C8000CDBFCF91DF911F910F91FF90EF90DF903B
:100C9000CF90BF90AF909F908F907F906F905F901C
:100CA0004F903F902F900895EF92FF920F931F93D4
:100CB000CF93DF93EC017A018B0177FF0FC0E881BE
:100CC000F9810190F081E02D6DE209951095009574
:100CD000F094E094E11CF11C011D111D2AE0B80103
:100CE000A701CE010E94BC05DF91CF911F910F910A
:100CF000FF90EF9008950F931F938C01AB0166272F
:100D000057FD6095762F0E945406C8010E94A505E4
:100D10001F910F9108951F920F920FB60F921124F9
:100D20002F933F934F935F936F937F938F939F93F3
:100D3000AF93BF93EF93FF9380917F0190918001D8
:100D4000892B29F0E0917F01F09180010995FF91B5
:100D5000EF91BF91AF919F918F917F916F915F9133
:100D60004F913F912F910F900FBE0F901F901895AC
:100D70001F920F920FB60F9211242F933F934F9310
:100D80005F936F937F938F939F93AF93BF93EF93F3
:100D9000FF938091810190918201892B29F0E0914C
:100DA0008101F09182010995FF91EF91BF91AF917F
:100DB0009F918F917F916F915F914F913F912F9173
:100DC0000F900FBE0F901F9018951F920F920FB6A5
:100DD0000F9211242F938F939F93AF93BF93809182
:100DE000830190918401A0918501B09186010196C3
:100DF000A11DB11D8093830190938401A09385016F
:100E0000B09386018091870190918801A09189011A
:100E1000B0918A018050904CAF4FBF4F80938701B3
:100E200090938801A0938901B0938A0127C0809193
:100E3000870190918801A0918901B0918A01805821
:100E40009E43A040B0408093870190938801A09377
:100E50008901B0938A0180918B0190918C01A091BE
:100E60008D01B0918E010196A11DB11D80938B0162
:100E700090938C01A0938D01B0938E018091870196
:100E800090918801A0918901B0918A0181589E4377
:100E9000A040B04060F6BF91AF919F918F912F918C
:100EA0000F900FBE0F901F9018958FB7F894209158
:100EB0008B0130918C0140918D0150918E018FBF3B
:100EC000B901CA010895EF92FF920F931F937B011E
:100ED0008C018FB7F89440918B0150918C016091F7
:100EE0008D0170918E018FBF2FB7F89480918B0187
:100EF00090918C01A0918D01B0918E012FBF841B28
:100F0000950BA60BB70BE816F9060A071B0760F747
:100F10001F910F91FF90EF900895789484B58260AF
:100F200084BD84B5816084BD85B5826085BD85B58D
:100F3000816085BDEEE6F0E0808181608083E1E83C
:100F4000F0E0808182608083808181608083E0E83E
:100F5000F0E0808181608083E1EBF0E0808184605B
:100F60008083E0EBF0E0808181608083EAE7F0E05D
:100F700080818460808380818260808380818160C1
:100F800080838081806880831092C10008951F93C0
:100F9000CF93DF93182FEB0161E00E941F08E12F30
:100FA000F0E0E156FF4F8491833051F4809180004E
:100FB000806880938000D0938900C09388003BC0F4
:100FC000843051F480918000806280938000D093BF
:100FD0008B00C0938A002FC0813039F4209729F10B
:100FE00084B5806884BDC7BD26C0823039F420979F
:100FF000E1F084B5806284BDC8BD1DC0863041F477
:101000008091B00080688093B000C093B30013C09B
:10101000873041F48091B00080628093B000C0932B
:10102000B40009C0C038D10514F460E001C061E02B
:10103000812F0E943D08DF91CF911F910895282FA5
:1010400030E0C90185579F4FFC01949129583F4FCB
:10105000F9018491882381F0E82FF0E0E859FF4FEF
:10106000E491F0E0662329F48081909589238083C0
:1010700008958081892B80830895482F50E0CA010C
:1010800081569F4FFC012491CA0185579F4FFC0157
:10109000949149585F4FFA0134913323C1F12223CF
:1010A00031F1233021F4809180008F7705C0243006
:1010B00031F4809180008F7D8093800018C02130B2
:1010C00019F484B58F7704C0223021F484B58F7D64
:1010D00084BD0DC0263021F48091B0008F7705C00B
:1010E000273029F48091B0008F7D8093B000E32FEA
:1010F000F0E0E359FF4FE491F0E0662329F48081AA
:1011000090958923808308958081892B8083089519
:10111000482F50E0CA0181569F4FFC012491CA011B
:1011200085579F4FFC01949149585F4FFA013491C4
:10113000332319F420E030E035C0222331F123308D
:1011400021F4809180008F7705C0243031F48091A4
:1011500080008F7D8093800018C0213019F484B501
:101160008F7704C0223021F484B58F7D84BD0DC0FB
:10117000263021F48091B0008F7705C0273029F404
:101180008091B0008F7D8093B000E32FF0E0EE58A7
:10119000FF4FE491F0E0808120E030E0892311F0FE
:1011A00021E030E0C9010895EF92FF920F931F9361
:1011B0007B018C0122E030E040E050E00E94D60943
:1011C000205C3D4B404F5F4FCA01B901A801970118
:1011D0000E94D609C901DA010197A109B109292F95
:1011E0003A2F4B2F552747FD5A950196A11DB11D4A
:1011F0002093C50081508093C400E1ECF0E0808131
:101200008061808380818860808380818068808322
:101210001F910F91FF90EF900895982F8091C0003B
:1012200085FFFCCF9093C600089580918F01909127
:10123000900180589F4F2091910130919201821B23
:10124000930B60E870E00E94A1090895409191011C
:101250005091920180918F01909190018417950790
:1012600019F42FEF3FEF0FC0FA01ED56FE4F20812A
:10127000CA01019660E870E00E94A1099093920172
:101280008093910130E0C90108951F920F920FB62B
:101290000F9211242F933F934F935F936F937F93FC
:1012A0008F939F93AF93BF93EF93FF934091C600AB
:1012B000E0918F01F0919001CF01019660E870E01C
:1012C0000E94A1099C01809191019091920128179F
:1012D000390739F0ED56FE4F40833093900120934B
:1012E0008F01FF91EF91BF91AF919F918F917F916E
:1012F0006F915F914F913F912F910F900FBE0F9083
:101300001F901895629FD001739FF001829FE00D9E
:10131000F11D649FE00DF11D929FF00D839FF00D74
:10132000749FF00D659FF00D9927729FB00DE11D20
:10133000F91F639FB00DE11DF91FBD01CF011124FD
:10134000089597FB092E07260AD077FD04D049D0CF
:1013500006D000201AF4709561957F4F0895F6F736
:10136000909581959F4F0895A1E21A2EAA1BBB1B51
:10137000FD010DC0AA1FBB1FEE1FFF1FA217B30761
:10138000E407F50720F0A21BB30BE40BF50B661F77
:10139000771F881F991F1A9469F76095709580953B
:1013A00090959B01AC01BD01CF01089597FB092EDB
:1013B00005260ED057FD04D0D7DF0AD0001C38F424
:1013C00050954095309521953F4F4F4F5F4F089571
:1013D000F6F790958095709561957F4F8F4F9F4F51
:1013E0000895AA1BBB1B51E107C0AA1FBB1FA6176C
:1013F000B70710F0A61BB70B881F991F5A95A9F7BE
:1014000080959095BC01CD010895EE0FFF1F0590CA
:0A141000F491E02D0994F894FFCF49
:10141A00486F6C612C20736F7920656C20726F6243
:10142A006F74206E756D65726F200008000B0004E2
:10143A000002000E000F0010001100030005000753
:0C144A000009000A00000000007E050000
:00000001FF
